:1000000012C077C029C028C027C026C025C024C080
:1000100023C022C021C021C01FC01EC01DC01CC0E3
:100020001BC01AC019C011241FBECFEDCDBF10E0F8
:10003000A0E6B0E0E0ECF7E002C005900D92A23738
:10004000B107D9F710E0A2E7B0E001C01D92AC37CC
:10005000B107E1F722D1B2C3D3CF1F920F920FB6EF
:100060000F9211248F939F93EF93FF93DF93CF937E
:1000700000D0CDB7DEB7E6E3F0E08081882F90E0D6
:1000800081709070882319F081E08A8301C01A8200
:10009000E6E3F0E08081882F90E082709070009716
:1000A00019F081E0898301C0198290917B008A81D7
:1000B000981779F08A81813061F08981813021F04F
:1000C00081E080937A0002C010927A0081E08093F0
:1000D00079008A8180937B000F900F90CF91DF9100
:1000E000FF91EF919F918F910F900FBE0F901F90F6
:1000F00018951F920F920FB60F9211242F938F9382
:100100009F93EF93FF93DF93CF9300D000D00F9294
:10011000CDB7DEB71A8219821D821CC0E0E3F0E081
:100120008081882F90E084709070009719F081E0B2
:100130008D8301C01D8289819A8101969A8389836A
:1001400089819A812EE08131920720F081E08D83B0
:1001500081E08C838D81882309F38C81813009F4BF
:100160008BC01A8219821BC0E0E3F0E08081882FE7
:1001700090E084709070009719F081E08D8301C049
:100180001D8289819A8101969A83898389819A81C6
:1001900027E08930920718F01D8281E08C838D81E1
:1001A000813011F389819A8123E08438920730F4F9
:1001B00081E08C8380917700809378008C818130FE
:1001C00009F45AC01B8250C01A82198219C0E0E398
:1001D000F0E08081882F90E084709070009719F093
:1001E00081E08D8301C01D8289819A8101969A8365
:1001F000898389819A81823E910510F081E08D8307
:100200008D81882321F31A82198219C0E0E3F0E07E
:100210008081882F90E084709070009719F081E0C1
:100220008D8301C01D8289819A8101969A83898379
:1002300089819A8122E0843A920708F01D828D819B
:10024000813021F380917800880F80937800898134
:100250009A81823E910528F0809178008F5F80938B
:1002600078008B818F5F8B838B81803208F4ACCFD9
:1002700080917800809377000F900F900F900F90EF
:100280000F90CF91DF91FF91EF919F918F912F91DF
:100290000F900FBE0F901F901895DF93CF930F9282
:1002A000CDB7DEB7E7E3F0E08CEF8083E8E3F0E082
:1002B00083E08083E1E3F0E08BEB8083E2E3F0E036
:1002C00084E48083E5E5F0E082E08083A5E5B0E0AA
:1002D000E5E5F0E080818E7F8C93EBE5F0E080E453
:1002E0008083E0E4F0E083E08083ABE5B0E0EBE521
:1002F000F0E0808180628C937894E0E5F0E081E822
:100300008083E3E5F0E081E08083EFE4F0E081EAE0
:100310008083EEE4F0E081E0808354D18CE661D10B
:1003200080917900813051F4109279004BD1809105
:100330007A00813011F417D201C02AD2E0E3F0E054
:100340008081882F90E0807490700097B1F43AD14A
:10035000809176008C3619F48DE643D102C08CE68C
:1003600040D1E0E3F0E08081882F90E080749070CD
:100370000097B9F38FEF9FEF08D180917800882321
:1003800009F499C080917800809378001BD1809106
:1003900078008F3509F4FCD1809178008F3D09F405
:1003A000E2D1809178008F3111F48DE61AD18091DD
:1003B00078008F3911F48CE614D1809178008F3653
:1003C00011F488E40ED1809178008F3411F481E427
:1003D00008D180917800873511F48AE302D18091A9
:1003E0007800873611F482E3FCD08091780087375B
:1003F00011F48BE2F6D0809178008F3E11F484E204
:10040000F0D0809178008F3C11F48DE1EAD080919A
:100410007800873D11F485E1E4D080917800873E33
:1004200011F48EE0DED080917800873F11F487E0F0
:10043000D8D0809178008F3A11F480E0D2D08091AA
:1004400078008F3811F485E6CCD080917800873918
:1004500011F48EE5C6D080917800873A11F486E5D4
:10046000C0D080917800873B11F48FE4BAD080919E
:1004700078008F3211F48DE6B4D080917800873304
:1004800019F481E08093720080917800873119F42B
:1004900081E080937300809178008F3019F481E0BF
:1004A0008093740080917800873219F481E0809302
:1004B00075001092780080917200813021F468D12B
:1004C0008FEF9FEF62D080917300813069F480914B
:1004D000760089838CE685D08FEF9FE456D08981A2
:1004E00080D08FEF9FE451D080917400813099F5D6
:1004F000E8E4F0E080818F5F8083E8E4F0E08081D1
:10050000813031F5E8E4F0E0808181508083EAE4D5
:10051000F0E080818F5F8083EAE4F0E080818130C9
:10052000B9F4EAE4F0E0808181508083E6E5F0E010
:1005300080818F5F8083E6E5F0E08081813041F447
:10054000E8E4F0E081E08083EAE4F0E081E08083A9
:100550008FEF94E01AD080917500813009F0E0CEE1
:10056000809176008C5E80937600809176008C3648
:1005700028F0809176008B568093760080917600EB
:1005800030D08FEF9FEA01D0CBCEDF93CF9300D056
:100590000F92CDB7DEB79A8389831B8289819A81B6
:1005A000009711F081E08B8389819A8101979A836A
:1005B00089838B81882389F70F900F900F90CF91BB
:1005C000DF910895DF93CF93CDB7DEB7109272001D
:1005D000109273001092740010927500CF91DF9109
:1005E0000895DF93CF930F92CDB7DEB789838981CA
:1005F000823188F4E8E4F0E01082AAE4B0E0898176
:10060000882F90E0FC01E05AFF4F80818C93E6E553
:10061000F0E08FEF808389818231C0F0898184325C
:10062000A8F4E8E4F0E01082EAE4F0E08FEF8083E1
:10063000A6E5B0E08981282F30E083E290E0821BBC
:10064000930BFC01E05AFF4F80818C9389818432A7
:10065000A8F08981863390F4A8E4B0E08981882FDE
:1006600090E08497FC01E05AFF4F80818C93EAE48C
:10067000F0E08FEF8083E6E5F0E010828981863339
:10068000C0F089818834A8F4E8E4F0E08FEF80833B
:10069000AAE4B0E08981282F30E087E490E0821B53
:1006A000930BFC01E05AFF4F80818C93E6E5F0E06C
:1006B000108289818834B0F089818A3598F4E8E421
:1006C000F0E08FEF8083EAE4F0E01082A6E5B0E08E
:1006D0008981882F90E088549040FC01E05AFF4FB8
:1006E00080818C9389818A35C0F089818C36A8F409
:1006F000A8E4B0E08981282F30E08BE690E0821BEF
:10070000930BFC01E05AFF4F80818C93EAE4F0E008
:100710001082E6E5F0E08FEF808389818C3661F40A
:1007200028E430E0AAE4B0E0E6E5F0E01082808161
:100730008C938C91F901808389818D3669F428E44A
:1007400030E0AAE4B0E0E6E5F0E081EE808380816D
:100750008C938C91F90180838981809376000F902E
:10076000CF91DF910895DF93CF93CDB7DEB780911E
:1007700076008F5F80937600809176008C3610F043
:1007800010927600809176002CDFCF91DF91089552
:10079000DF93CF93CDB7DEB7809176008150809301
:1007A0007600809176008B3F18F08BE68093760080
:1007B0008091760016DFCF91DF910895F894FFCFF6
:1007C000000F1E2D3C4B5A69788796A5B4C3D2E121
:0207D000F0FF38
:00000001FF
